******************************************************************************
                  TI ARM Linker PC v15.12.5                    
******************************************************************************
>> Linked Tue Oct 31 17:54:27 2017

OUTPUT FILE NAME:   <TMS570LS_FEE_0432.out>
ENTRY POINT SYMBOL: "_c_int00"  address: 0000c8e8


MEMORY CONFIGURATION

         name            origin    length      used     unused   attr    fill
----------------------  --------  ---------  --------  --------  ----  --------
  VECTORS               00000000   00000020  00000020  00000000     X
  FLASH0                00000020   0005ffe0  0000f260  00050d80  R  X
  STACKS                08000000   00001500  00000000  00001500  RW  
  RAM                   08001500   00006b00  00000275  0000688b  RW  


SEGMENT ALLOCATION MAP

run origin  load origin   length   init length attrs members
----------  ----------- ---------- ----------- ----- -------
00000000    00000000    0000f284   0000f284    r-x
  00000000    00000000    00000020   00000020    r-x .intvecs
  00000020    00000020    0000d774   0000d774    r-x .text
  0000d794    0000d794    00001848   00001848    r-x FEE_TEXT_SECTION
  0000efdc    0000efdc    00000180   00000180    r-- .const
  0000f15c    0000f15c    000000d0   000000d0    r-- FEE_CONST_SECTION
  0000f230    0000f230    00000054   00000054    r-- .cinit
08001500    08001500    00000276   00000000    rw-
  08001500    08001500    00000129   00000000    rw- FEE_DATA_SECTION
  0800162a    0800162a    000000ca   00000000    rw- .bss
  080016f4    080016f4    00000082   00000000    rw- .data


SECTION ALLOCATION MAP

 output                                  attributes/
section   page    origin      length       input sections
--------  ----  ----------  ----------   ----------------
.intvecs   0    00000000    00000020     
                  00000000    00000020     sys_intvecs.obj (.intvecs)

.text      0    00000020    0000d774     
                  00000020    00005904     ti_fee_util.obj (.text)
                  00005924    000024f0     sys_selftest.obj (.text)
                  00007e14    00001750     ti_fee_ini.obj (.text)
                  00009564    00001018     ti_fee_main.obj (.text)
                  0000a57c    00000a64     system.obj (.text)
                  0000afe0    00000898     sys_vim.obj (.text)
                  0000b878    000005e8     esm.obj (.text)
                  0000be60    00000340     sys_core.obj (.text)
                  0000c1a0    0000027c     sys_main.obj (.text)
                  0000c41c    0000026c     sys_vim.obj (.text:retain)
                  0000c688    00000260     F021_API_CortexR4_BE.lib : FlashStateMachine.InitializeFlashBanks.obj (.text:Fapi_initializeFlashBanks)
                  0000c8e8    00000208     sys_startup.obj (.text:retain)
                  0000caf0    0000017c     F021_API_CortexR4_BE.lib : FlashStateMachine.SetActiveBank.obj (.text:Fapi_setActiveFlashBank)
                  0000cc6c    00000150     pinmux.obj (.text)
                  0000cdbc    00000110     sys_pmu.obj (.text)
                  0000cecc    000000ec     esm.obj (.text:retain)
                  0000cfb8    000000e8     dabort.obj (.text)
                  0000d0a0    0000009c     rtsv7R4_T_be_eabi.lib : memcpy_t2.obj (.text)
                  0000d13c    00000094     F021_API_CortexR4_BE.lib : BlankCheck.obj (.text:Fapi_doBlankCheck)
                  0000d1d0    00000080                              : FlashStateMachine.EnableEepromSectors.obj (.text:Fapi_enableEepromBankSectors)
                  0000d250    0000007c     notification.obj (.text)
                  0000d2cc    0000007a     rtsv7R4_T_be_eabi.lib : memset_t2.obj (.text)
                  0000d346    00000002                           : startup.obj (.text)
                  0000d348    00000070                           : autoinit.obj (.text)
                  0000d3b8    0000006a                           : copy_decompress_rle.obj (.text)
                  0000d422    0000005e     F021_API_CortexR4_BE.lib : Read.LoopDword.obj (.text:_Fapi_loopRegionForValue)
                  0000d480    00000050                              : FlashStateMachine.Hercules.IsEccAddress.obj (.text:Fapi_isAddressEcc)
                  0000d4d0    00000050     rtsv7R4_T_be_eabi.lib : exit.obj (.text)
                  0000d520    0000004c                           : cpy_tbl.obj (.text)
                  0000d56c    00000044     F021_API_CortexR4_BE.lib : FlashStateMachine.EnableEepromSectors.obj (.text:_Fapi_EnableSectors)
                  0000d5b0    0000003c                              : FlashStateMachine.IssueFsmCommand.obj (.text:_Fapi_issueFsmCommand)
                  0000d5ec    00000036                              : Utilities.CalculateFletcher.obj (.text:Fapi_calculateFletcherChecksum)
                  0000d622    00000002     --HOLE-- [fill = 0]
                  0000d624    00000030                              : Async.WithAddress.obj (.text:Fapi_issueAsyncCommandWithAddress)
                  0000d654    00000030                              : Utilities.WaitDelay.obj (.text:Fapi_waitDelay)
                  0000d684    0000002c                              : Read.Common.obj (.text:_Fapi_readDword)
                  0000d6b0    0000002a                              : Async.obj (.text:Fapi_issueAsyncCommand)
                  0000d6da    00000022                              : Read.FlushPipeline.obj (.text:Fapi_flushPipeline)
                  0000d6fc    0000001c                              : FlashStateMachine.InitializeFlashBanks.obj (.text:_Fapi_divideUnsignedLong)
                  0000d718    00000014     rtsv7R4_T_be_eabi.lib : _lock.obj (.text)
                  0000d72c    00000010     F021_API_CortexR4_BE.lib : Utilities.GetNumberOfSectors.obj (.text:Fapi_getNumberOfBankSectors)
                  0000d73c    00000010                              : FlashStateMachine.ScaleFclk.obj (.text:_scaleEEFclk)
                  0000d74c    00000010                              : FlashStateMachine.ScaleFclk.obj (.text:_scaleMainFclk)
                  0000d75c    0000000e     rtsv7R4_T_be_eabi.lib : copy_decompress_none.obj (.text:decompress:none)
                  0000d76a    0000000c     F021_API_CortexR4_BE.lib : Read.WdService.obj (.text:_Fapi_checkWdService)
                  0000d776    00000002     --HOLE-- [fill = 0]
                  0000d778    00000008     Fapi_UserDefinedFunctions.obj (.text)
                  0000d780    00000006     rtsv7R4_T_be_eabi.lib : copy_decompress_rle.obj (.text:decompress:rle24)
                  0000d786    00000002     --HOLE-- [fill = 0]
                  0000d788    00000004     sys_phantom.obj (.text:retain)
                  0000d78c    00000008     Fapi_UserDefinedFunctions.obj (.tramp.Fapi_serviceWatchdogTimer.1)

FEE_TEXT_SECTION 
*          0    0000d794    00001848     
                  0000d794    00000cb4     ti_fee_writeAsync.obj (FEE_TEXT_SECTION)
                  0000e448    000007a4     ti_fee_read.obj (FEE_TEXT_SECTION)
                  0000ebec    000003f0     ti_fee_invalidateblock.obj (FEE_TEXT_SECTION)

.const     0    0000efdc    00000180     
                  0000efdc    00000180     sys_vim.obj (.const:s_vim_init)

FEE_CONST_SECTION 
*          0    0000f15c    000000d0     
                  0000f15c    00000084     Device_TMS570LS04.obj (FEE_CONST_SECTION)
                  0000f1e0    0000004c     ti_fee_cfg.obj (FEE_CONST_SECTION)

.cinit     0    0000f230    00000054     
                  0000f230    00000017     (.cinit..data.load) [load image, compression = rle]
                  0000f247    00000001     --HOLE-- [fill = 0]
                  0000f248    0000000b     (.cinit.FEE_DATA_SECTION.load) [load image, compression = rle]
                  0000f253    00000005     --HOLE-- [fill = 0]
                  0000f258    00000009     (.cinit..bss.load) [load image, compression = rle]
                  0000f261    00000003     --HOLE-- [fill = 0]
                  0000f264    00000008     (__TI_handler_table)
                  0000f26c    00000018     (__TI_cinit_table)

FEE_DATA_SECTION 
*          0    08001500    00000129     UNINITIALIZED
                  08001500    000000f7     ti_fee_ini.obj (FEE_DATA_SECTION)
                  080015f7    00000001     ti_fee_main.obj (FEE_DATA_SECTION)
                  080015f8    00000028     ti_fee_util.obj (FEE_DATA_SECTION:uninit)
                  08001620    00000009     ti_fee_util.obj (FEE_DATA_SECTION:init)

.bss       0    0800162a    000000ca     UNINITIALIZED
                  0800162a    00000064     (.common:SpecialRamBlock)
                  0800168e    00000064     (.common:SpecialRamBlock2)
                  080016f2    00000002     (.common:Status)

.data      0    080016f4    00000082     UNINITIALIZED
                  080016f4    00000064     sys_main.obj (.data:read_data)
                  08001758    0000000c     rtsv7R4_T_be_eabi.lib : exit.obj (.data:$O1$$)
                  08001764    00000008                           : _lock.obj (.data:$O1$$)
                  0800176c    00000008     F021_API_CortexR4_BE.lib : FlashStateMachine.ScaleFclk.obj (.data)
                  08001774    00000001                              : FlashStateMachine.SetActiveBank.obj (.data)
                  08001775    00000001     sys_main.obj (.data)

MODULE SUMMARY

       Module                                        code    ro data   rw data
       ------                                        ----    -------   -------
    .\source\
       ti_fee_util.obj                               22788   0         49     
       sys_selftest.obj                              9456    0         0      
       ti_fee_ini.obj                                5968    0         247    
       ti_fee_main.obj                               4120    0         1      
       ti_fee_writeAsync.obj                         3252    0         0      
       sys_vim.obj                                   2820    384       0      
       system.obj                                    2660    0         0      
       ti_fee_read.obj                               1956    0         0      
       esm.obj                                       1748    0         0      
       ti_fee_invalidateblock.obj                    1008    0         0      
       sys_main.obj                                  636     0         303    
       sys_core.obj                                  832     0         0      
       sys_startup.obj                               520     0         0      
       pinmux.obj                                    336     0         0      
       sys_pmu.obj                                   272     0         0      
       dabort.obj                                    232     0         0      
       Device_TMS570LS04.obj                         0       132       0      
       notification.obj                              124     0         0      
       ti_fee_cfg.obj                                0       76        0      
       sys_intvecs.obj                               32      0         0      
       Fapi_UserDefinedFunctions.obj                 16      0         0      
       sys_phantom.obj                               4       0         0      
    +--+---------------------------------------------+-------+---------+---------+
       Total:                                        58780   592       600    
                                                                              
    C:/ti/Hercules/F021 Flash API/02.01.01/F021_API_CortexR4_BE.lib
       FlashStateMachine.InitializeFlashBanks.obj    636     0         0      
       FlashStateMachine.SetActiveBank.obj           380     0         1      
       FlashStateMachine.EnableEepromSectors.obj     196     0         0      
       BlankCheck.obj                                148     0         0      
       Read.LoopDword.obj                            94      0         0      
       FlashStateMachine.Hercules.IsEccAddress.obj   80      0         0      
       FlashStateMachine.IssueFsmCommand.obj         60      0         0      
       Utilities.CalculateFletcher.obj               54      0         0      
       Async.WithAddress.obj                         48      0         0      
       Utilities.WaitDelay.obj                       48      0         0      
       Read.Common.obj                               44      0         0      
       Async.obj                                     42      0         0      
       FlashStateMachine.ScaleFclk.obj               32      0         8      
       Read.FlushPipeline.obj                        34      0         0      
       Utilities.GetNumberOfSectors.obj              16      0         0      
       Read.WdService.obj                            12      0         0      
    +--+---------------------------------------------+-------+---------+---------+
       Total:                                        1924    0         9      
                                                                              
    C:/ti/ccsv7/tools/compiler/ti-cgt-arm_15.12.5.LTS/lib/rtsv7R4_T_be_eabi.lib
       memcpy_t2.obj                                 156     0         0      
       memset_t2.obj                                 122     0         0      
       autoinit.obj                                  112     0         0      
       copy_decompress_rle.obj                       112     0         0      
       exit.obj                                      80      0         12     
       cpy_tbl.obj                                   76      0         0      
       _lock.obj                                     20      0         8      
       copy_decompress_none.obj                      14      0         0      
       startup.obj                                   2       0         0      
    +--+---------------------------------------------+-------+---------+---------+
       Total:                                        694     0         20     
                                                                              
       Linker Generated:                             0       75        0      
    +--+---------------------------------------------+-------+---------+---------+
       Grand Total:                                  61398   667       629    


LINKER GENERATED COPY TABLES

__TI_cinit_table @ 0000f26c records: 3, size/record: 8, table size: 24
	.data: load addr=0000f230, load size=00000017 bytes, run addr=080016f4, run size=00000082 bytes, compression=rle
	FEE_DATA_SECTION: load addr=0000f248, load size=0000000b bytes, run addr=08001500, run size=00000129 bytes, compression=rle
	.bss: load addr=0000f258, load size=00000009 bytes, run addr=0800162a, run size=000000ca bytes, compression=rle


LINKER GENERATED HANDLER TABLE

__TI_handler_table @ 0000f264 records: 2, size/record: 4, table size: 8
	index: 0, handler: __TI_decompress_rle24
	index: 1, handler: __TI_decompress_none

VENEERS

callee name               veneer name
   callee addr  veneer addr  call addr  call info
--------------  -----------  ---------  ----------------
Fapi_serviceWatchdogTimer  $Ven$TA$L$PI$$Fapi_serviceWatchdogTimer
   0000d778     0000d78c     0000d770   F021_API_CortexR4_BE.lib : Read.WdService.obj (.text:_Fapi_checkWdService)

[1 trampolines]
[1 trampoline calls]


GLOBAL SYMBOLS: SORTED ALPHABETICALLY BY Name 

address   name                                    
-------   ----                                    
0000d4d1  C$$EXIT                                 
0000f15c  Device_FlashDevice                      
0000d5ed  Fapi_calculateFletcherChecksum          
0000d13d  Fapi_doBlankCheck                       
0000d1d1  Fapi_enableEepromBankSectors            
0000d6db  Fapi_flushPipeline                      
0000d72d  Fapi_getNumberOfBankSectors             
0000c689  Fapi_initializeFlashBanks               
0000d481  Fapi_isAddressEcc                       
0000d6b1  Fapi_issueAsyncCommand                  
0000d625  Fapi_issueAsyncCommandWithAddress       
0000d778  Fapi_serviceWatchdogTimer               
0000caf1  Fapi_setActiveFlashBank                 
0000d655  Fapi_waitDelay                          
0000f1ec  Fee_BlockConfiguration                  
0000f1e0  Fee_VirtualSectorConfiguration          
UNDEFED   SHT$$INIT_ARRAY$$Base                   
UNDEFED   SHT$$INIT_ARRAY$$Limit                  
0800162a  SpecialRamBlock                         
0800168e  SpecialRamBlock2                        
080016f2  Status                                  
00000a64  TI_FeeInternal_AlignAddressForECC       
000010e8  TI_FeeInternal_BlankCheck               
00005154  TI_FeeInternal_CheckForError            
00002bd8  TI_FeeInternal_CheckModuleState         
00002c38  TI_FeeInternal_CheckReadParameters      
000057f8  TI_FeeInternal_EnableRequiredFlashSector
000031dc  TI_FeeInternal_FeeManager               
00000e34  TI_FeeInternal_FindNextVirtualSector    
000052d4  TI_FeeInternal_Fletcher16               
00001eb8  TI_FeeInternal_GetArrayIndex            
00001e00  TI_FeeInternal_GetBlockIndex            
00001dcc  TI_FeeInternal_GetBlockNumber           
00000df4  TI_FeeInternal_GetBlockSize             
00002d68  TI_FeeInternal_GetCurrentBlockAddress   
00001e78  TI_FeeInternal_GetDataSetIndex          
00002e6c  TI_FeeInternal_GetNextFlashAddress      
00001bf0  TI_FeeInternal_GetVirtualSectorIndex    
00000020  TI_FeeInternal_GetVirtualSectorParameter
00004d2c  TI_FeeInternal_InvalidateErase          
00000d78  TI_FeeInternal_PollFlashStatus          
00002ebc  TI_FeeInternal_SanityCheck              
000030b0  TI_FeeInternal_SetClearCopyBlockState   
00004fe8  TI_FeeInternal_StartProgramBlock        
00002014  TI_FeeInternal_UpdateBlockOffsetArray   
000046d8  TI_FeeInternal_WriteBlockHeader         
00000664  TI_FeeInternal_WriteDataF021            
00000a9c  TI_FeeInternal_WriteInitialize          
00004a40  TI_FeeInternal_WritePreviousBlockHeader 
000001b8  TI_FeeInternal_WriteVirtualSectorHeader 
00005400  TI_Fee_ErrorRecovery                    
080015f6  TI_Fee_FapiInitCalled                   
000050e4  TI_Fee_GetStatus                        
08001500  TI_Fee_GlobalVariables                  
00007e94  TI_Fee_Init                             
0000ebec  TI_Fee_InvalidateBlock                  
00009564  TI_Fee_MainFunction                     
0000e448  TI_Fee_Read                             
000056c4  TI_Fee_SuspendResumeErase               
0000d794  TI_Fee_WriteAsync                       
080015e1  TI_Fee_bEraseSuspended                  
080015e2  TI_Fee_oStatusWord                      
080015dc  TI_Fee_u32ActCpyVS                      
080015d4  TI_Fee_u32BlockEraseCount               
080015d0  TI_Fee_u32FletcherChecksum              
080015cc  TI_Fee_u8DataSets                       
080015d8  TI_Fee_u8DeviceIndex                    
080015e0  TI_Fee_u8ErrEraseVS                     
080015e6  TI_FlashStatusWord                      
0000d56d  _Fapi_EnableSectors                     
0000d76b  _Fapi_checkWdService                    
0000d5b1  _Fapi_issueFsmCommand                   
0000d423  _Fapi_loopRegionForValue                
0000d685  _Fapi_readDword                         
0000f26c  __TI_CINIT_Base                         
0000f284  __TI_CINIT_Limit                        
0000f264  __TI_Handler_Table_Base                 
0000f26c  __TI_Handler_Table_Limit                
0000c198  __TI_PINIT_Base                         
0000c19c  __TI_PINIT_Limit                        
0000d349  __TI_auto_init                          
08001758  __TI_cleanup_ptr                        
0000d75d  __TI_decompress_none                    
0000d781  __TI_decompress_rle24                   
0800175c  __TI_dtors_ptr                          
08001760  __TI_enable_exit_profile_output         
ffffffff  __TI_pprof_out_hndl                     
ffffffff  __TI_prof_data_size                     
ffffffff  __TI_prof_data_start                    
00000000  __TI_static_base__                      
0000d2cd  __aeabi_memclr                          
0000d2cd  __aeabi_memclr4                         
0000d2cd  __aeabi_memclr8                         
0000d0a1  __aeabi_memcpy                          
0000d0a1  __aeabi_memcpy4                         
0000d0a1  __aeabi_memcpy8                         
0000d2cf  __aeabi_memset                          
0000d2cf  __aeabi_memset4                         
0000d2cf  __aeabi_memset8                         
ffffffff  __binit__                               
ffffffff  __c_args__                              
0000c8e8  _c_int00                                
0000c0a8  _coreClearAuxiliaryDataFault_           
0000c0c4  _coreClearAuxiliaryInstructionFault_    
0000c070  _coreClearDataFaultAddress_             
0000c038  _coreClearDataFault_                    
0000c08c  _coreClearInstructionFaultAddress_      
0000c054  _coreClearInstructionFault_             
0000bf9c  _coreDisableEventBusExport_             
0000c000  _coreDisableFlashEcc_                   
0000bfcc  _coreDisableRamEcc_                     
0000bf84  _coreEnableEventBusExport_              
0000bfe4  _coreEnableFlashEcc_                    
0000c018  _coreEnableIrqVicOffset_                
0000bfb4  _coreEnableRamEcc_                      
0000c0a0  _coreGetAuxiliaryDataFault_             
0000c0bc  _coreGetAuxiliaryInstructionFault_      
0000c068  _coreGetDataFaultAddress_               
0000c030  _coreGetDataFault_                      
0000c084  _coreGetInstructionFaultAddress_        
0000c04c  _coreGetInstructionFault_               
0000be60  _coreInitRegisters_                     
0000bf18  _coreInitStackPointer_                  
0000cfb8  _dabort                                 
0000c0e0  _disable_FIQ_interrupt_                 
0000c0e8  _disable_IRQ_interrupt_                 
0000c0d8  _disable_interrupt_                     
0000c0f0  _enable_interrupt_                      
0000c180  _errata_CORTEXR4_66_                    
0000c0f8  _esmCcmErrorsClear_                     
0000bf64  _getCPSRValue_                          
0000bf6c  _gotoCPUIdle_                           
08001764  _lock                                   
0000d727  _nop                                    
0000ce28  _pmuDisableCountersGlobal_              
0000ce10  _pmuEnableCountersGlobal_               
0000cea4  _pmuGetCycleCount_                      
0000ceac  _pmuGetEventCount_                      
0000ceb8  _pmuGetOverflow_                        
0000cdbc  _pmuInit_                               
0000ce70  _pmuResetCounters_                      
0000ce40  _pmuResetCycleCounter_                  
0000ce58  _pmuResetEventCounters_                 
0000ce98  _pmuSetCountEvent_                      
0000ce88  _pmuStartCounters_                      
0000ce90  _pmuStopCounters_                       
0000d71f  _register_lock                          
0000d719  _register_unlock                        
0000d73d  _scaleEEFclk                            
0000d74d  _scaleMainFclk                          
0000d347  _system_post_cinit                      
08001768  _unlock                                 
0000d4d5  abort                                   
00006908  adc1ParityCheck                         
ffffffff  binit                                   
000069c0  can1ParityCheck                         
00006a9c  can2ParityCheck                         
00005934  ccmSelfCheck                            
00007938  ccmr4GetConfigValue                     
0000623c  checkB0RAMECC                           
0000642c  checkB1RAMECC                           
00006f08  checkClockMonitor                       
0000661c  checkFlashECC                           
00006fdc  checkFlashEEPROMECC                     
00007184  checkPLL1Slip                           
000072a0  checkRAMAddrParity                      
00006cc0  checkRAMECC                             
000073a8  checkRAMUERRTest                        
000060c0  checkefcSelfTest                        
0000d521  copy_in                                 
00005b38  cpuSelfTest                             
00006700  cpuSelfTestFail                         
000066f8  custom_dabort                           
0000c1a0  delay                                   
00007d28  disableParity                           
00005f64  efcCheck                                
0000789c  efcGetConfigValue                       
00006098  efcSelfTest                             
00005fec  efcStuckZeroTest                        
00007cd4  enableParity                            
000079b4  errata_PBIST_4                          
0000ba04  esmActivateNormalOperation              
0000bae8  esmClearStatus                          
0000bb34  esmClearStatusBuffer                    
0000b9c8  esmDisableError                         
0000ba40  esmDisableInterrupt                     
0000b99c  esmEnableError                          
0000ba14  esmEnableInterrupt                      
0000bc34  esmEnterSelfTest                        
0000b980  esmError                                
0000bd0c  esmGetConfigValue                       
0000bb70  esmGetStatus                            
0000bbfc  esmGetStatusBuffer                      
0000d250  esmGroup1Notification                   
0000d260  esmGroup2Notification                   
0000cecc  esmHighInterrupt                        
0000b878  esmInit                                 
0000bcbc  esmSelfTestStatus                       
0000bb50  esmSetCounterPreloadValue               
0000ba6c  esmSetInterruptLevel                    
0000b9f4  esmTriggerErrorPinReset                 
0000d4dd  exit                                    
00007504  fmcBus1ParityCheck                      
00006160  fmcBus2Check                            
0000619c  fmcECCcheck                             
0000d2b8  gioNotification                         
000067b0  het1ParityCheck                         
00006850  htu1ParityCheck                         
0000c1cc  main                                    
0000a6a8  mapClocks                               
0000d0a1  memcpy                                  
00005a78  memoryInit                              
0000d270  memoryPort0TestFailNotification         
0000d28c  memoryPort1TestFailNotification         
0000d2d5  memset                                  
00006b64  mibspi1ParityCheck                      
0000cc6c  muxInit                                 
08001775  oResult                                 
00007630  pbistFail                               
000076b4  pbistGetConfigValue                     
00005eac  pbistIsTestCompleted                    
00005ed8  pbistIsTestPassed                       
00005f0c  pbistPortTestStatus                     
00005db0  pbistRun                                
00005bd0  pbistSelfCheck                          
00005e7c  pbistStop                               
0000a654  periphInit                              
0000d788  phantomInterrupt                        
0000ccf4  pinmuxGetConfigValue                    
080016f4  read_data                               
00000000  resetEntry                              
0000d2a8  rtiNotification                         
00005924  selftestFailNotification                
0000a614  setupFlash                              
0000a57c  setupPLL                                
0000adf4  sramGetConfigValue                      
000077fc  stcGetConfigValue                       
00005abc  stcSelfCheck                            
000066fc  stcSelfCheckFail                        
0000a888  systemGetConfigValue                    
0000a78c  systemInit                              
0000a858  systemPowerDown                         
0000ac48  tcmflashGetConfigValue                  
0000a5cc  trimLPO                                 
0000b0b4  vimChannelMap                           
0000b2b0  vimDisableInterrupt                     
0000b158  vimEnableInterrupt                      
0000b334  vimGetConfigValue                       
0000afe0  vimInit                                 
00006704  vimParityCheck                          
0000c41c  vimParityErrorHandler                   


GLOBAL SYMBOLS: SORTED BY Symbol Address 

address   name                                    
-------   ----                                    
00000000  __TI_static_base__                      
00000000  resetEntry                              
00000020  TI_FeeInternal_GetVirtualSectorParameter
000001b8  TI_FeeInternal_WriteVirtualSectorHeader 
00000664  TI_FeeInternal_WriteDataF021            
00000a64  TI_FeeInternal_AlignAddressForECC       
00000a9c  TI_FeeInternal_WriteInitialize          
00000d78  TI_FeeInternal_PollFlashStatus          
00000df4  TI_FeeInternal_GetBlockSize             
00000e34  TI_FeeInternal_FindNextVirtualSector    
000010e8  TI_FeeInternal_BlankCheck               
00001bf0  TI_FeeInternal_GetVirtualSectorIndex    
00001dcc  TI_FeeInternal_GetBlockNumber           
00001e00  TI_FeeInternal_GetBlockIndex            
00001e78  TI_FeeInternal_GetDataSetIndex          
00001eb8  TI_FeeInternal_GetArrayIndex            
00002014  TI_FeeInternal_UpdateBlockOffsetArray   
00002bd8  TI_FeeInternal_CheckModuleState         
00002c38  TI_FeeInternal_CheckReadParameters      
00002d68  TI_FeeInternal_GetCurrentBlockAddress   
00002e6c  TI_FeeInternal_GetNextFlashAddress      
00002ebc  TI_FeeInternal_SanityCheck              
000030b0  TI_FeeInternal_SetClearCopyBlockState   
000031dc  TI_FeeInternal_FeeManager               
000046d8  TI_FeeInternal_WriteBlockHeader         
00004a40  TI_FeeInternal_WritePreviousBlockHeader 
00004d2c  TI_FeeInternal_InvalidateErase          
00004fe8  TI_FeeInternal_StartProgramBlock        
000050e4  TI_Fee_GetStatus                        
00005154  TI_FeeInternal_CheckForError            
000052d4  TI_FeeInternal_Fletcher16               
00005400  TI_Fee_ErrorRecovery                    
000056c4  TI_Fee_SuspendResumeErase               
000057f8  TI_FeeInternal_EnableRequiredFlashSector
00005924  selftestFailNotification                
00005934  ccmSelfCheck                            
00005a78  memoryInit                              
00005abc  stcSelfCheck                            
00005b38  cpuSelfTest                             
00005bd0  pbistSelfCheck                          
00005db0  pbistRun                                
00005e7c  pbistStop                               
00005eac  pbistIsTestCompleted                    
00005ed8  pbistIsTestPassed                       
00005f0c  pbistPortTestStatus                     
00005f64  efcCheck                                
00005fec  efcStuckZeroTest                        
00006098  efcSelfTest                             
000060c0  checkefcSelfTest                        
00006160  fmcBus2Check                            
0000619c  fmcECCcheck                             
0000623c  checkB0RAMECC                           
0000642c  checkB1RAMECC                           
0000661c  checkFlashECC                           
000066f8  custom_dabort                           
000066fc  stcSelfCheckFail                        
00006700  cpuSelfTestFail                         
00006704  vimParityCheck                          
000067b0  het1ParityCheck                         
00006850  htu1ParityCheck                         
00006908  adc1ParityCheck                         
000069c0  can1ParityCheck                         
00006a9c  can2ParityCheck                         
00006b64  mibspi1ParityCheck                      
00006cc0  checkRAMECC                             
00006f08  checkClockMonitor                       
00006fdc  checkFlashEEPROMECC                     
00007184  checkPLL1Slip                           
000072a0  checkRAMAddrParity                      
000073a8  checkRAMUERRTest                        
00007504  fmcBus1ParityCheck                      
00007630  pbistFail                               
000076b4  pbistGetConfigValue                     
000077fc  stcGetConfigValue                       
0000789c  efcGetConfigValue                       
00007938  ccmr4GetConfigValue                     
000079b4  errata_PBIST_4                          
00007cd4  enableParity                            
00007d28  disableParity                           
00007e94  TI_Fee_Init                             
00009564  TI_Fee_MainFunction                     
0000a57c  setupPLL                                
0000a5cc  trimLPO                                 
0000a614  setupFlash                              
0000a654  periphInit                              
0000a6a8  mapClocks                               
0000a78c  systemInit                              
0000a858  systemPowerDown                         
0000a888  systemGetConfigValue                    
0000ac48  tcmflashGetConfigValue                  
0000adf4  sramGetConfigValue                      
0000afe0  vimInit                                 
0000b0b4  vimChannelMap                           
0000b158  vimEnableInterrupt                      
0000b2b0  vimDisableInterrupt                     
0000b334  vimGetConfigValue                       
0000b878  esmInit                                 
0000b980  esmError                                
0000b99c  esmEnableError                          
0000b9c8  esmDisableError                         
0000b9f4  esmTriggerErrorPinReset                 
0000ba04  esmActivateNormalOperation              
0000ba14  esmEnableInterrupt                      
0000ba40  esmDisableInterrupt                     
0000ba6c  esmSetInterruptLevel                    
0000bae8  esmClearStatus                          
0000bb34  esmClearStatusBuffer                    
0000bb50  esmSetCounterPreloadValue               
0000bb70  esmGetStatus                            
0000bbfc  esmGetStatusBuffer                      
0000bc34  esmEnterSelfTest                        
0000bcbc  esmSelfTestStatus                       
0000bd0c  esmGetConfigValue                       
0000be60  _coreInitRegisters_                     
0000bf18  _coreInitStackPointer_                  
0000bf64  _getCPSRValue_                          
0000bf6c  _gotoCPUIdle_                           
0000bf84  _coreEnableEventBusExport_              
0000bf9c  _coreDisableEventBusExport_             
0000bfb4  _coreEnableRamEcc_                      
0000bfcc  _coreDisableRamEcc_                     
0000bfe4  _coreEnableFlashEcc_                    
0000c000  _coreDisableFlashEcc_                   
0000c018  _coreEnableIrqVicOffset_                
0000c030  _coreGetDataFault_                      
0000c038  _coreClearDataFault_                    
0000c04c  _coreGetInstructionFault_               
0000c054  _coreClearInstructionFault_             
0000c068  _coreGetDataFaultAddress_               
0000c070  _coreClearDataFaultAddress_             
0000c084  _coreGetInstructionFaultAddress_        
0000c08c  _coreClearInstructionFaultAddress_      
0000c0a0  _coreGetAuxiliaryDataFault_             
0000c0a8  _coreClearAuxiliaryDataFault_           
0000c0bc  _coreGetAuxiliaryInstructionFault_      
0000c0c4  _coreClearAuxiliaryInstructionFault_    
0000c0d8  _disable_interrupt_                     
0000c0e0  _disable_FIQ_interrupt_                 
0000c0e8  _disable_IRQ_interrupt_                 
0000c0f0  _enable_interrupt_                      
0000c0f8  _esmCcmErrorsClear_                     
0000c180  _errata_CORTEXR4_66_                    
0000c198  __TI_PINIT_Base                         
0000c19c  __TI_PINIT_Limit                        
0000c1a0  delay                                   
0000c1cc  main                                    
0000c41c  vimParityErrorHandler                   
0000c689  Fapi_initializeFlashBanks               
0000c8e8  _c_int00                                
0000caf1  Fapi_setActiveFlashBank                 
0000cc6c  muxInit                                 
0000ccf4  pinmuxGetConfigValue                    
0000cdbc  _pmuInit_                               
0000ce10  _pmuEnableCountersGlobal_               
0000ce28  _pmuDisableCountersGlobal_              
0000ce40  _pmuResetCycleCounter_                  
0000ce58  _pmuResetEventCounters_                 
0000ce70  _pmuResetCounters_                      
0000ce88  _pmuStartCounters_                      
0000ce90  _pmuStopCounters_                       
0000ce98  _pmuSetCountEvent_                      
0000cea4  _pmuGetCycleCount_                      
0000ceac  _pmuGetEventCount_                      
0000ceb8  _pmuGetOverflow_                        
0000cecc  esmHighInterrupt                        
0000cfb8  _dabort                                 
0000d0a1  __aeabi_memcpy                          
0000d0a1  __aeabi_memcpy4                         
0000d0a1  __aeabi_memcpy8                         
0000d0a1  memcpy                                  
0000d13d  Fapi_doBlankCheck                       
0000d1d1  Fapi_enableEepromBankSectors            
0000d250  esmGroup1Notification                   
0000d260  esmGroup2Notification                   
0000d270  memoryPort0TestFailNotification         
0000d28c  memoryPort1TestFailNotification         
0000d2a8  rtiNotification                         
0000d2b8  gioNotification                         
0000d2cd  __aeabi_memclr                          
0000d2cd  __aeabi_memclr4                         
0000d2cd  __aeabi_memclr8                         
0000d2cf  __aeabi_memset                          
0000d2cf  __aeabi_memset4                         
0000d2cf  __aeabi_memset8                         
0000d2d5  memset                                  
0000d347  _system_post_cinit                      
0000d349  __TI_auto_init                          
0000d423  _Fapi_loopRegionForValue                
0000d481  Fapi_isAddressEcc                       
0000d4d1  C$$EXIT                                 
0000d4d5  abort                                   
0000d4dd  exit                                    
0000d521  copy_in                                 
0000d56d  _Fapi_EnableSectors                     
0000d5b1  _Fapi_issueFsmCommand                   
0000d5ed  Fapi_calculateFletcherChecksum          
0000d625  Fapi_issueAsyncCommandWithAddress       
0000d655  Fapi_waitDelay                          
0000d685  _Fapi_readDword                         
0000d6b1  Fapi_issueAsyncCommand                  
0000d6db  Fapi_flushPipeline                      
0000d719  _register_unlock                        
0000d71f  _register_lock                          
0000d727  _nop                                    
0000d72d  Fapi_getNumberOfBankSectors             
0000d73d  _scaleEEFclk                            
0000d74d  _scaleMainFclk                          
0000d75d  __TI_decompress_none                    
0000d76b  _Fapi_checkWdService                    
0000d778  Fapi_serviceWatchdogTimer               
0000d781  __TI_decompress_rle24                   
0000d788  phantomInterrupt                        
0000d794  TI_Fee_WriteAsync                       
0000e448  TI_Fee_Read                             
0000ebec  TI_Fee_InvalidateBlock                  
0000f15c  Device_FlashDevice                      
0000f1e0  Fee_VirtualSectorConfiguration          
0000f1ec  Fee_BlockConfiguration                  
0000f264  __TI_Handler_Table_Base                 
0000f26c  __TI_CINIT_Base                         
0000f26c  __TI_Handler_Table_Limit                
0000f284  __TI_CINIT_Limit                        
08001500  TI_Fee_GlobalVariables                  
080015cc  TI_Fee_u8DataSets                       
080015d0  TI_Fee_u32FletcherChecksum              
080015d4  TI_Fee_u32BlockEraseCount               
080015d8  TI_Fee_u8DeviceIndex                    
080015dc  TI_Fee_u32ActCpyVS                      
080015e0  TI_Fee_u8ErrEraseVS                     
080015e1  TI_Fee_bEraseSuspended                  
080015e2  TI_Fee_oStatusWord                      
080015e6  TI_FlashStatusWord                      
080015f6  TI_Fee_FapiInitCalled                   
0800162a  SpecialRamBlock                         
0800168e  SpecialRamBlock2                        
080016f2  Status                                  
080016f4  read_data                               
08001758  __TI_cleanup_ptr                        
0800175c  __TI_dtors_ptr                          
08001760  __TI_enable_exit_profile_output         
08001764  _lock                                   
08001768  _unlock                                 
08001775  oResult                                 
ffffffff  __TI_pprof_out_hndl                     
ffffffff  __TI_prof_data_size                     
ffffffff  __TI_prof_data_start                    
ffffffff  __binit__                               
ffffffff  __c_args__                              
ffffffff  binit                                   
UNDEFED   SHT$$INIT_ARRAY$$Base                   
UNDEFED   SHT$$INIT_ARRAY$$Limit                  

[251 symbols]
